:020000040000FA
:100000000A128A11142A8207003400341A34003488
:100010002934003435340034413400344D34003454
:1000200059340034633400346D3400347634003491
:100030008034003489340034933400349D340034E7
:10004000A6340034B2340034BF340034C834003431
:10005000CF340034D9340034E5340034EF34003484
:10006000F834003405340134113401341A340134C5
:1000700024340134303401343A340134433401340B
:100080004F34013459340134653401346F34013450
:100090007834013484340134903401349A34013496
:1000A000A6340134B0340134BE340134CA340134CE
:1000B000D6340134E0340134EE340134FD340134FB
:1000C0000934023417340234243402343034023414
:1000D0003C3402344A340234593402346534023434
:1000E00073340234823402348E3402349C34023449
:1000F000AB340234BB340234C8340234D834023452
:10010000E7340234F3340234063403341534033450
:100110002634033437340334473403345834033437
:10012000693403347A3403348D340334A334033410
:10013000B7340334C9340334DB340334EE340334CA
:10014000FE34033418340434323404344434043474
:1001500060340434663404348034043482073F3419
:1001600006345B344F3466346D347D3407347F3469
:0E0170006F3477347C3439345E347934713432
:1002000082078034043492340434B0340434C43467
:100210000434CE340434E83404340B3405341C3450
:1002200005343F3405345A3405346A3405348D348A
:100230000534A7340534C1340534EC3405340E34A8
:10024000063429340634403406345D3406348034B0
:100250000634A2340634CC340634F03406341B346D
:10026000073447340734693407348C340734B734DF
:100270000734E4340734FD3407343134083453345C
:10028000083476340834AA340834DE34083412349E
:1002900009344634093483340934B0340934EC3435
:1002A000093432340A346E340A34A0340A34E63461
:1002B0000A3418340B345E340B34A4340B34F43465
:1002C0000B344E340C3497340C34D0340C34163494
:1002D0000D3470340D34CA340D342E340E349C3445
:1002E0000E34E2340E344B340F34D2340F344034F5
:1002F0001034AE341034263411348A34113420349E
:100300001234C03412344234133414341434963456
:1003100014345434153412341634DA341634983410
:100320001734743418346E34193472341A349434E3
:100330001B34CA341C34CE341D342C341F34803466
:10034000203424342234D2342334D03425349C3421
:100350002734B83429341030A8000310A40DA50D9B
:100360000310A00DA10D031CBB292308A50722081B
:10037000A4070318A50AA80BAD2908001030A8008F
:10038000A201A3010310A60DA70D0310A00DA10D3E
:10039000A20DA30D23082502031DD0292208240243
:1003A0000319D4290318DB292508A3022408A20273
:1003B000031CA3032614A80BC2290800AB00831357
:1003C000633084000430A80000088403000403198B
:1003D000ED298403A80BE42908002A088000840A78
:1003E0002B0880000800AB0083135C308400640895
:1003F000840784072A088000840A2B08800084036D
:10040000E408031D072A0430E40084078407E4039A
:1004100084030008840300040319002A840A0008E6
:100420008A00840300088200E301E201E101E001A7
:10043000DF01DE01DD01DC01E4010508C30006087F
:10044000C4000708C5008F3083160F0570388F0071
:10045000831203179E019F0103139F0183169F01BF
:100460008312031799019A01552ABD003D0803190B
:10047000080001303D02031D422A00000000000078
:1004800000000800BD0300000000BE01502A8312D6
:1004900003130330A0000A128A11A00B4D2ABE0AD2
:1004A0003E083D02031D472A0800831605148514E3
:1004B0000616061707148714071507160511861266
:1004C00087110717861783120313E5016508C30018
:1004D00043088500E6016608C40044088600E70179
:1004E0006708C50045088700831681139501803091
:1004F000831203179500942A83168712FF30920007
:10050000043083129200133083169200F830831265
:1005100012058316CB0004304B0483129200123074
:1005200095000C30970008000313AC01AD01AE013B
:100530007A2C5030AC005030AD007930AE0008005D
:100540003830AC00BF30AD00AE0108003830AC0030
:100550007730AD003930AE000800793083120313D4
:10056000AC005430AD005E30AE00080003304602EF
:10057000031DBC2AE73045020319C02A0318332B98
:1005800064308312A400A501831645088312A000DD
:10059000831646088312A100BE2183120313260886
:1005A0008316C900831227088316CA0000308A0008
:1005B00049088A11AE2083120313AE006430A400F0
:1005C000A501831645088312A000831646088312EE
:1005D000A1008A11BE218312031322088316C700CB
:1005E000831223088316C8000A308312A400A501D1
:1005F000831647088312A000831648088312A100BF
:100600008A11BE218312031326088316C9008312A0
:1006100027088316CA0000308A0049088A11AE20D4
:1006200083120313AD000A30A400A5018316470806
:100630008312A000831648088312A1008A11BE21EC
:100640008312031322088316C7008312230883161C
:10065000C80000308A0047088A11AE2083120313B5
:10066000AC00AE17080027304602031D392B0F30AF
:10067000450203193D2B0318C92BE8308312A4004F
:100680000330A500831645088312A0008316460890
:100690008312A100BE218312031326088316C9000A
:1006A000831227088316CA0000308A0049088A117D
:1006B000AE2083120313AE00E830A4000330A5007F
:1006C000831645088312A000831646088312A100F2
:1006D0008A11BE218312031322088316C7008312D6
:1006E00023088316C80064308312A400A501831672
:1006F00047088312A000831648088312A1008A11BC
:10070000BE218312031326088316C900831227080B
:100710008316CA0000308A0049088A11AE2083126D
:100720000313AD006430A400A501831647088312AB
:10073000A000831648088312A1008A11BE218312EB
:10074000031322088316C700831223088316C800E8
:100750000A308312A400A501831647088312A00063
:10076000831648088312A1008A11BE218312031345
:1007700026088316C900831227088316CA00003092
:100780008A0049088A11AE2083120313AC00AD170A
:10079000080010308312A4002730A50083164508F6
:1007A0008312A000831646088312A100BE21831283
:1007B000031326088316C900831227088316CA006C
:1007C00000308A0049088A11AE2083120313AE005C
:1007D0001030A4002730A500831645088312A0001E
:1007E000831646088312A1008A11BE2183120313C7
:1007F00022088316C700831223088316C800E83036
:100800008312A4000330A500831647088312A000BA
:10081000831648088312A1008A11BE218312031394
:1008200026088316C900831227088316CA000030E1
:100830008A0049088A11AE2083120313AD00E83004
:10084000A4000330A500831647088312A000831676
:1008500048088312A1008A11BE21831203132208C3
:100860008316C700831223088316C80064308312DE
:10087000A400A501831647088312A0008316480828
:100880008312A1008A11BE21831203132608831646
:10089000C900831227088316CA0000308A0049085D
:1008A0008A11AE2083120313AC00AC1708000F307E
:1008B0004205C40000308A004408AE2083120313AE
:1008C000AC008316420E0F39C40000308A00440881
:1008D0008A11AE2083120313AD000F308316430537
:1008E000C40000308A0044088A11AE20831203132A
:1008F000AE0008005910C601E12DC100831607158E
:100900000616071485140514061707168714831294
:10091000591C922CC60A643046020319922C031803
:10092000922C08004108031DB42C831607110130D6
:1009300083122C05C2004208C412031DC4164408C9
:10094000860001302D05C20042084311031D4315E6
:100950004308850001302E05C2004208C511031D61
:10096000C51545088700080001304102031DD72C3A
:1009700083160612023083122C05C2004208C412EC
:10098000031DC4164408860002302D05C20042082B
:100990004311031D43154308850002302E05C20094
:1009A0004208C511031DC51545088700080002301F
:1009B0004102031DFA2C83160710043083122C0504
:1009C000C2004208C412031DC41644088600043045
:1009D0002D05C20042084311031D4315430885003D
:1009E00004302E05C2004208C511031DC515450877
:1009F0008700080003304102031D1D2D831685105A
:100A0000083083122C05C2004208C412031DC4160C
:100A10004408860008302D05C20042084311031D1A
:100A200043154308850008302E05C2004208C51151
:100A3000031DC51545088700080004304102031D49
:100A4000402D83160510103083122C05C200420879
:100A5000C412031DC4164408860010302D05C200C0
:100A600042084311031D43154308850010302E052D
:100A7000C2004208C511031DC515450887000800BE
:100A800005304102031D632D8316061320308312A7
:100A90002C05C2004208C412031DC4164408860077
:100AA00020302D05C20042084311031D43154308A1
:100AB000850020302E05C2004208C511031DC51552
:100AC00045088700080006304102031D862D831665
:100AD0000712403083122C05C2004208C412031DC5
:100AE000C4164408860040302D05C2004208431158
:100AF000031D43154308850040302E05C2004208FF
:100B0000C511031DC51545088700080007304102BF
:100B1000031DA82D83168710803083122C05C20078
:100B20004208C412031DC4164408860080302D05F7
:100B3000C20042084311031D43154308850080305D
:100B40002E05C2004208C511031DC51545088700C2
:100B50000800831203134014BF01831203138A1188
:100B6000401CBE2D3F087D2483120313BF0A0830AA
:100B70003F028A110319BF014010CC2DC011C018CB
:100B8000C42D0F18C015C62D0F1CC015C01DCC2DAF
:100B9000C0100F18C0144014D030AA000530F3293B
:100BA0008A11AD2D0330831203179F008F308316F7
:100BB00003131F0550389F0083121F139F171F1424
:100BC0000800AF01B001B101B201B301B401272E99
:100BD000831203138A119F18212E83161E08831275
:100BE000BB001E08BC002F08A0003008A10031087F
:100BF000A2003208A3003B08A0073C0803183C0FE2
:100C0000A1070030FE0003187E0FA2070030FE008F
:100C100003187E0FA3072008AF002108B0002208A8
:100C2000B1002308B200B30A0319B40AC3301F0588
:100C300020389F0001303522831203139F148A113C
:100C4000E82D2530AA000630F3298A11E82DC701C6
:100C5000C801C901CA018D2E831247088316BA0044
:100C6000831248088316BB00831249088316BC0010
:100C700083124A088316BD00831247088316BE00FC
:100C8000831248088316BF00831249088316C000E8
:100C900083124A088316C1003A08BE023B08031CAF
:100CA0003B0FBF023C08031C3C0FC0023D08031C65
:100CB0003D0FC1023E088312C70083163F0883120E
:100CC000C800831640088312C900831641088312A6
:100CD000CA00831638088312C70783163908FE0036
:100CE000831203187E0FC8070030FE0003187E0F22
:100CF000C9070030FE0003187E0FCA074708831695
:100D0000BA00831248088316BB003A088312A00079
:100D100083163B088312A1000800B501B601B70194
:100D2000D9145911D9115912D9125913FE2E8312FF
:100D300003133A10591B9F2E8F1B3A14A12E8F1F9D
:100D40003A143A1CAA2E8F1BA72E5913A82E5917F6
:100D5000B50AB60A08008312031339105919B32EC5
:100D60000F183914B52E0F1C3914391CD52E0F1835
:100D7000BB2E5911BC2E5915B910D918C22E861B7D
:100D8000B914C42E861FB914B91CD42EB70A043066
:100D900037020319D52E031CD52E861BD12ED91050
:100DA000D22ED914B7010800B7010800AB26831270
:100DB00003138A11D918E62ED91159160F303602AD
:100DC0000319E72E031CE72ED916E72EB6013815B6
:100DD000591AD91C3811381DF02ED9155912D912AB
:100DE00008008A1197268A11D626FC308312031335
:100DF000AA0006308A11F3298A11F12ED913CB01EA
:100E0000CC018A15A2280030831203133302A000FC
:100E1000013034022004031D752F0310320C831699
:100E2000B2008312310C8316B1008312300C83168A
:100E3000B00083122F0C8316AF0004308312A00081
:100E400003108316B20CB10CB00CAF0C8312A00BC4
:100E5000202F83162F08B8003008B9002C268312E3
:100E6000031320088316B400831221088316B500EB
:100E7000B601B7018312B301B401AF01B001B101F2
:100E8000B2014C08831635028A11031D4B2F8312C1
:100E90004B0883163402B3100319502F0318B314F0
:100EA00001303407AF000030031801303507B000BF
:100EB00083124C0883163002031D622F83124B08E5
:100EC00083162F0233110319672F031C3315B31137
:100ED000B31C3319B315B31D752F34088312CB001F
:100EE000831635088312CC00D91708000F3022056D
:100EF000A9000310230C8312A1008316220C831275
:100F0000A0000330A2000310A10CA00CA20B832FA1
:100F100020088316A400543024028A1503191528CA
:100F200003181528240AAA0003102A0DAB00031089
:100F3000240DAC0000308A002B088A110320831294
:100F40000313A000013083162B078A11032083129C
:100F50000313A10000308A0083162C088A11032095
:100F600083120313A200013083162C078A11032079
:100F700083120313A300230821028316A600831201
:100F8000220820028316A500031CA603250883124D
:100F9000A000831626088312A10083162908831255
:100FA000A200A3018A11AB21831203132408831624
:100FB000AA00831225088316AB0003102B0CA8008F
:100FC0002A0CA70003308312A00003108316A80C7C
:100FD000A70C83128A11A00BE52F03108316240D92
:100FE000AA0000308A002A08032083120313A000FD
:100FF000013083162A078A11032083120313A100EC
:1010000083162808831221078316AC002708831251
:1010100020078316AB000318AC0A2B088312A0002C
:1010200083162C088312A1000800240AAA00543059
:101030002A02AB0003102B0DAC0054302402AD008B
:1010400003102D0DAE0001308A002C088A110021FA
:1010500083120313A000013083162C078A1100218C
:1010600083120313A10001308A0083162E088A110F
:10107000002183120313A200013083162E078A1168
:10108000002183120313A300230821028316A60064
:101090008312220820028316A500031CA60325083C
:1010A0008312A000831626088312A1008316290844
:1010B0008312A200A3018A11AB2183120313240817
:1010C0008316AA00831225088316AB0003102B0C8D
:1010D000A8002A0CA70003308312A0000310831677
:1010E000A80CA70C83128A15A00B6E285430831607
:1010F0002402AA0003102A0DAB0001308A002B083D
:101100008A11002183120313A000013083162B07DC
:101110008A11002183120313A10083162808831269
:1011200021078316AD002708831220078316AC0021
:101130000318AD0A2C088312A00083162D08831211
:10114000A1000800CD01CE01CF01D001D101D20113
:10115000D301D401D501D6015D29831203134C08B4
:101160005602031DB5284B0855020319B928031868
:10117000BB288A11A02A4C085402031DC1284B0821
:1011800053020319C728031CC7288A11992A05305E
:1011900035026F11031D03186F15EF15D91B6F1D55
:1011A000EF11EF1D212954084C028316A100831270
:1011B00053084B028316A000031CA1032008A200C1
:1011C0002108A3008A117627831203132008CD007B
:1011D0002108CE004E0850028A15031DF1284D0843
:1011E0004F020319F52803180B2950084E028316E5
:1011F000A10083124F084D028316A000031CA10317
:101200002008C5002108C6008A11B62283120313E4
:1012100059108A151F294E0850028316A100831207
:101220004D084F028316A000031CA1032008C5002F
:101230002108C6008A11B622831203135914D91348
:10124000B501080083120313EE006E0803178D002A
:1012500083168C130C1483120C080800EC006D0824
:1012600003178C0003136C0803178D0083168C136F
:101270000C1555308D00AA308D008C140C118C1873
:101280003F2908000030222183120313EA000130B5
:101290008A15222183120313EB006A08A0006B0851
:1012A000A10008006808ED0000302E21831203130E
:1012B0006908ED0001308A152E29DB108A117C2285
:1012C0008A11D2253530831203139000F130AA0021
:1012D00006308A11DE21A93083120313AA000530DB
:1012E0008A11DE21E83083120313AA0005308A1127
:1012F000DE218A154221831203132008D30021081E
:10130000D400530854048A150319DB148312031301
:101310003508031D92299030AA0009308A11F3295B
:101320008A1586295A11591EDB185A155A1D252A65
:101330008A11A622831203135914A230AA0009307D
:101340008A11F32983120313DA11D91DDB18DA1578
:101350008A15DA1D9D29D911B130AA0009308A11E8
:10136000F329831203135A12D91DD91A5A168A1552
:101370005A1EAC295910DA12D91EDB18DA16DA1EF9
:10138000252AC630AA0009308A11F32983120313D3
:101390005A13D91DDB185A178A155A1FC129D9119A
:1013A000AF01B0010130B100B201C701C801C901EC
:1013B000CA01B3010130B4008A1103278312031359
:1013C00052084C02D80051084B02D700031CD80326
:1013D00057088316C200831258088316C3008A1167
:1013E00057248312031351085204DA170319DA132E
:1013F0005B14D91ADA1F5B108A155B1C172A510877
:10140000E8005208E90052218A11AD220D30831202
:101410000313AA000A308A11F329831203138A15D1
:10142000D91D062A5108D3005208D400252AD91DF7
:101430001E2AD9114B08D1004C08D2002330AA0033
:101440000A308A11F3298A15DC290A305407D6009C
:1014500080305307D5000318D60A0310530DAF0090
:10146000540DB0000430FE000310AF0DB00DFE0BA4
:10147000342AB101B2015308C7005408C800C90199
:10148000CA01B3010130B4008A1103278A15AD20C7
:10149000831203138A15D91D532AD9114D08CF0081
:1014A0004E08D000D9175830AA000A308A11F32903
:0414B0008A15442A2B
:02400E00D433A9
:0442000000000000BA
:00000001FF
